:020000020000FC
:1000000055CD0000000000001FC0A5C193C0000036
:1000100000009DC000000000000000000203040674
:10002000080C10182030406080000406080C1018DE
:100030002030406080A0C00000070F1F3F00050572
:100040000D050305030302004FB662FD0EC05520E7
:1000500009F00994C52DC095089483FDC795C4BDCA
:10006000C093A10064604FBE1895C09164000894CD
:1000700083FDC795C4BDC093A1006B7FC091640090
:10008000CF3F09F420C070FF02C082FD05C04FBE03
:10009000C19897989598189575FD0EC065FD0CC090
:1000A000C091B300C0FD9298C1FD9398C2FD949891
:1000B000CAEFC095CA95F1F7C19897989598209284
:1000C000A1004FBE189524BCCC27C064C8BF646093
:1000D000F6CFC0CF70FFBECF65FDBCCFC19ABACFFF
:1000E00070FFB8CF65FDB6CF979AB4CF70FFB2CF8F
:1000F00065FDB0CF959AAECF929A70FFABCF65FDFC
:10010000A9CFC7E0CA95F1F7C19AA4CF939A70FF1F
:10011000A1CF65FD9FCFC7E0CA95F1F7979A9ACF17
:10012000949A70FF97CF65FD95CFC7E0CA95F1F718
:10013000959A90CF4FB6C9B7CF7EC9BF6E7FCCB569
:10014000CE0DDDB5DF1DDBBDCABD4FBE18953FB678
:100150008F7EA9B7A072A2118061A9B7AF7DA9BF98
:10016000A9B7AE7FA9BF7894A0916800AA2341F0F7
:1001700085FD2BC0A0916800AA95A093680025C0BA
:1001800040E050E085FD15C0A6B396FDA095A0FD0A
:100190004FEFAEB5A06496FDAF7BAEBDAA27A062BF
:1001A000A8BF8D7FA6B396FDA095A0FD5FEF451774
:1001B00039F7A8E161FDA093680085FD03C0A8E1BF
:1001C000A093680040939700816085FD0EC0A091C8
:1001D0006900AA2331F0A0916900AA95A093690053
:1001E00004C08061AA27A062A8BF80FF38C0A09188
:1001F00097004A2F61FF8E7F85FD18C0403F08F0B1
:1002000040EFA42FA295AF704A0F5091B800533021
:1002100069F0A695A69550FD01C0A69552FD03C0B4
:10022000A41B4A2F03C04A0F08F44FEFA091A0006F
:100230004A1708F44A2F40936100A72FA67079F05F
:10024000A0916D00A695A69556E0A50F509161006E
:10025000A50FA093610018F4AFEFA0936100A091E7
:100260006100A093630040916300A0919C004A1735
:1002700008F04A2F542EA091A200AA2309F422C00C
:10028000542F5A1B10F4A42F50E0BA2E8894AA1FA2
:10029000AA2EA091A400A095AA22A50E58F0A09184
:1002A000A300A21509F0AA95AA0EA093A30048F0F6
:1002B0004A2D08C0A091A300BA1608F0A395A093F8
:1002C000A3004FEF409364007F7D485F08F07062A9
:1002D000A52DA03408F06860A0916000A395A093BC
:1002E000600059F0F894A9B7A160A9BF84FF03C0CA
:1002F000A9B7A062A9BF3FBE1895A0917400A395AD
:10030000A093740041E050916800552329F085FFC7
:1003100003C05A9550936800A0919700A13018F03F
:1003200020929A000DC020929B002092A500A091DF
:100330009A00AF5FA0939A0018F0AFEFA0939A00D5
:10034000F894A9B7A160A9BF84FF03C0A9B7A062B0
:10035000A9BF3FBE18953FB646B557B58F7EA9B722
:10036000A072A2118061A9B7AF7DA9BFA9B7AE7F66
:10037000A9BF789481FD25C0AEB5AF7B96FDA06482
:10038000AEBD8260A6B396FDA095A0FF05C04093C8
:1003900065005093660041C1AEB5A06496FDAF7B89
:1003A000AEBDAA27A062A8BF8D7F85FF01C028C16E
:1003B00040E0A6B396FDA095A0FD22C14093970012
:1003C00011C1AEB5A06496FDAF7BAEBD8D7F61FF60
:1003D00072C0AEB5AF7B96FDA064AEBDAA27A06289
:1003E000A8BF82604093920050939300A090900029
:1003F0004A19B09091005B09BB24A22C4C385205DD
:1004000018F42092960049C0A091D600AA2359F171
:10041000483C520528F4A0E1BA2EAAE0AA2E23C037
:100420004836A1E05A0728F4A8E0BA2EAFE0AA2E79
:100430001AC0403DA2E05A0728F4A4E0BA2EAEE16B
:10044000AA2E11C0403AA5E05A0728F4A2E0BA2E1D
:10045000ACE3AA2E08C04839A8E05A0720F4A1E06E
:10046000BA2EA8E7AA2EC42EA0919400CA1AD52E9F
:10047000A0919500DA0ADD202AF4AFEFC094D09461
:10048000CA1ADA0A20929600A8E0A210A0E0CA14C4
:10049000DA0618F4A1E0A0939600409394005093DC
:1004A000950040919200509193004093900050939A
:1004B000910002E097C0A09165004A1BA0916600E0
:1004C0005A0B94FD82C093FD80C092FD7CC086FFD4
:1004D00003C0D52EC42E0CC05695479591FD73C010
:1004E0005695479590FD6FC0D52EC42ED694C794CF
:1004F00061FD19C0AC2DAC51AD2DA24008F005C076
:10050000DD2089F4AC2DA85C70F4A0916700A39560
:10051000AA2311F0A0936700AA3008F471C02092BA
:10052000970081606DC0A0916700AA2319F0AA9579
:10053000A0936700A22C5091BC0097FD06C0A0902C
:10054000CA00533011F4A090D200AAEFAA0EA22D37
:10055000A21DCA18DA0A4FB74170533049F4442338
:1005600021F087FD05C0806803C087FF01C08F7739
:10057000442359F0533031F4AFEFC094D094CA1AE9
:10058000DA0A03C040E050E020C0533049F4CC0CFC
:10059000DD1CAAE0CA1AD20818F4A0E0CA2ED22C98
:1005A000AFEFCA16D20418F04FEF50E00EC0A09182
:1005B000AE00CA9E412D000C441F50E008F012C04E
:1005C0004FEF50E00FC05695479594FF07C0552355
:1005D00009F04FEFA42FA6954A0F521D4F3F520529
:1005E00008F04FEF40939700816061FF09C0AFE1D1
:1005F000A095A923AB299A2F8F7DBB2009F4806297
:10060000A8E1A093680085FF03C0AAE0A09368005A
:1006100061FD03C085FD01C08F7E85FD03C0A6E09E
:10062000A0936900F894A9B7A160A9BF84FF03C093
:10063000A9B7A062A9BF3FBE189511E00AC013E098
:1006400008C01AE006C01EE104C014E602C018EC9F
:1006500000C005E1BB27BA95F1F70A95D9F71A95BD
:10066000C1F708952AE338E709C020E33CE806C053
:100670002AE234EB03C025E238EC00C012E095FD1D
:100680009F7D95FF9062BB27939ABA95F1F7979A51
:10069000BA95F1F79798BA95F1F79398BA95F1F75B
:1006A000C19AB091AF00BA95F1F7C198B7E8BA9581
:1006B000F1F71A9521F7022FB22FBA95F1F70A95A3
:1006C000D9F73A95D9F6939A0895221B39E0001F7D
:1006D0003A9509F40895221F211B18F4210F8894DC
:1006E000F6CF0894F4CF622C722CB0E08894B395C6
:1006F000221F331FE0F7379527958894912E802E7F
:10070000020B130B10F4192D082D10F4889401C05E
:100710000894661C771CBA9571F7172D062D08955D
:10072000322D11232AF43A9500951095031B130BD3
:10073000F894029F712C002D129F912C802C78949C
:10074000780C172D921C292DB4E06B2E2695179549
:1007500007956A94D9F7332321F000951095031B70
:10076000130B0895089510917B00169500917A005F
:100770000795B0917F00B01B0B2FB0918000B10B9B
:100780001B2F28F40038BFEF1B0740F009C00F37BC
:10079000120508F405C00FE710E002C000E81FEFE3
:1007A0000093840010938500089500918400B09117
:1007B00081000B0F10918500B09182001B1F20E07B
:1007C0003091850033230AF42A95B09183002B1FC2
:1007D0001AF4203F40F00AC02F3008F407C00FEF92
:1007E0001FEF2FE003C000E010E020EF3091630026
:1007F000B0919C003B1718F4323030F009C0B09132
:100800008500BB235AF004C0B0918500BB2332F4AD
:10081000009381001093820020938300089520911B
:10082000D80000918400000F10918500111F78DF1F
:1008300011232AF40038BFEF1B0740F009C00F371F
:10084000120508F405C00FE710E002C000E81FEF32
:10085000002352F0B0916200B01B0B2F18F0013052
:1008600008F00AC001E008C000950F5FB091620077
:100870000B0F08F001C00FEF009386000895209140
:10088000D90000918200109183004ADF11232AF4DD
:100890000130BFEF1B0740F009C00F3F120508F4FD
:1008A00005C00FEF10E002C001E01FEF112352F06E
:1008B000B0918600B01B0B2F18F0013008F00AC071
:1008C00001E008C000950F5FB09186000B0F08F0A3
:1008D00001C00FEF0093630008950FEF677F71FD74
:1008E00029C072FD09C06860B0917B00BA3020F069
:1008F000B52DB03408F4677FB091D500BB23D1F09B
:10090000B0917B00BB23B1F00FEF10917B00DDDED7
:10091000F894B091730072FDB5E00B9F112D002D7E
:100920007894112309F00FEFB0919F000B1710F48A
:1009300000919F0000939E00089500917A0010910D
:100940007B0000541140B0919E0010F4BA9501C094
:10095000B39511F0B0939E00089500C008952091C2
:10096000B700B6B1B6FDFBCF04B115B1B6B1BF77D4
:10097000B6B9B091AC00B395B093AC00B83060F1AB
:100980002092AC00B091D400BB2321F1112329F0B7
:10099000B091AD00BF3F61F009C0B091AD000B1741
:1009A00039F020F4BB2321F0BA9502C0B395E1F3EE
:1009B00000919C00B093AD00BA3F50F400ECB93FF9
:1009C00038F400E8B83F20F400E4B73F08F400E052
:1009D00000939C00777F0895B0919C00B39511F02F
:1009E000B0939C00B091AC00B73009F478600895E2
:1009F00002E3F894B091DA000B9F012D000C001F68
:100A00007894B0919C000B1710F000919C0000931B
:100A1000610000936300502E0093640000939F00D8
:100A2000089520927A00B0EFB0937B000895F89477
:100A30000CB51DB5209174007894309175006090CC
:100A400076000093750010937600031B160971FD64
:100A500003C076FD81C02BC0709077002093770093
:100A60002709222311F00FEF1FEF8090780090905C
:100A70007900309378006092790069181619109304
:100A80007C000091750010917600081919092091D9
:100A90007A0030917B0036952795020F131F10F4D2
:100AA0000FEF1FEF00937A0010937B0029C0209175
:100AB0007A0030917B003901B4E08B2EB2E09B2E9E
:100AC000343010F08A949A94383010F08A949A94C2
:100AD000769467948A94E1F726193709992021F0D2
:100AE000169507959A94E1F7200F311F20937A000D
:100AF00030937B0028F43FEF30937A0030937B00F3
:100B0000323008F4706471FF02C0B3E00DC0B091E0
:100B1000C60000917100023838F0B395003A08F031
:100B2000B395B63008F0B5E09B2EB4E08B2E109153
:100B30007B0000917A0024E0169507952A95E1F74D
:100B40000819120928F0B02FB250B12FB20910F4D1
:100B500002E010E0980126C020917A0030917B00DD
:100B600039017694679466946694669426193209DE
:100B700006950695200F321D20937A0030937B0056
:100B8000323008F07F7B04E036952795369527951F
:100B900026952695201B10F0223008F422E08901CA
:100BA0009090C60060FDFECFE0908C00F0908D002C
:100BB0006160B9B7B061B9BF380176FD44C07694C1
:100BC000679400938C0010938D00B92DB330E1F041
:100BD000B0FD04C0060D171D930106C0000F111FC4
:100BE0000250120922E030E0B92DB33068F02093B2
:100BF0008E0030938F0000938800109389006092DC
:100C00008A0070928B003DC000938E0010938F007D
:100C1000209388003093890060928A0070928B0044
:100C200071FF10C0B0916D00B33060F000918F0083
:100C300010917C001595010F28F022F020928E0073
:100C400000938F001EC0669400938C00B92DB330C2
:100C500091F0B0FD03C0060D262D03C0000F025019
:100C600022E0B92DB33038F020938E000093880035
:100C700060928A0006C000938E00209388006092E4
:100C80008A0000917D0002FD0350013029F495FD9A
:100C90000AC0B0E0B7B909C0023019F4B7E0B7B97B
:100CA00004C095FDF6CFB6E0B7B90091A400000FDF
:100CB00010F4BBE60B270093A40060FDFECFB2E06A
:100CC000B0936E006160B9B7B061B9BFB72FB670AD
:100CD000A1F020917A0030917B0036952795F89409
:100CE0000CB51DB5020F131F1BBD0ABD6160B0E13D
:100CF000B8BFB9B7B061B9BF789408956061209268
:100D00007E0020E067FD20E206C0606120927E0048
:100D100020E267FD20E0789401E076FD11C0B72F56
:100D2000B67009F06F7EB0917B00B55048F002E0DC
:100D3000B55020F003E0B55008F006E071FD0AE080
:100D400060FD12C0B0917E00BB2371F071FF08C03E
:100D5000B0916D00B33020F0B0916E00BA9519F4E7
:100D6000789470615CC0AEDF789400000000F89465
:100D700076FD16C010917B00173008F017E0B5E043
:100D80001B0F72FD10E183FF110F62FF110F71FD48
:100D900012E8B4B56090A100B61990F2B10B80F2E0
:100DA000B0B7B77FB0BFB8B1B0B7B860B0BFB0919F
:100DB0007E00B395B0937E00B8B176FD06C0B1E079
:100DC00071FDB2E0BA95F1F7B8B1B072B21709F09F
:100DD0001BC071FF05C003950A3008F00395B0CF22
:100DE00064FF99CF6F7E3CB56DB470907A008090AF
:100DF0007B00370D681C6BBC3ABD6160B0E1B8BFC9
:100E0000B9B7B061B9BF87CFB0916D00B23008F407
:100E100082CF64FD80CF0A9509F092CF7F7E20912A
:100E20008E0030918F00F894B0E1B8BF0CB51DB5BD
:100E3000020F131F1BBD0ABDE0908800F0908900CF
:100E40006160B9B7B061B9BF7894B72FB67039F0A7
:100E5000B0916D0072FFB395B0936D0009C074FF3F
:100E600007C067FD05C064FD03C0BF91BF91DEC42C
:100E7000089500E063FF03C064FF01C001E0F8943F
:100E800010917100B7E01B9F212D102D7894200F39
:100E90002695179526951795269517951093710009
:100EA000183718F4B8E7B093710000917100B09151
:100EB00072000B1720F06062C1989798959860FDBA
:100EC000FECFE0908A00F0908B006160B9B7B0610E
:100ED000B9BF0895B2E095FD07C0F894B0937D00C6
:100EE000939A92987894E5C0F894B0937D00939A81
:100EF00094987894DEC0B3E082FF24C095FD11C0C1
:100F000002E0F894B0937D00E6E8F0E00093B300CF
:100F10009598949A62FF02C0979A01C0939878942A
:100F2000C8C002E0F894B0937D00E6E8F0E00093DA
:100F3000B300C198929A62FF02C0979A01C0939839
:100F40007894B7C095FD0BC0F894B0937D00E0E7AE
:100F5000F0E0959862FF01C0979A7894AAC0F8943F
:100F6000B0937D00E0E7F0E0C19862FF01C0979A7E
:100F700078949FC0B4E095FD07C0F894B0937D00CD
:100F8000929A9498789495C0F894B0937D00949A2E
:100F9000929878948EC0B5E082FF24C095FD11C070
:100FA00001E0F894B0937D00ECE7F0E00093B3002B
:100FB0009798939A62FF02C0C19A01C09298789460
:100FC00078C004E0F894B0937D00E0E9F0E000938D
:100FD000B3009798939A62FF02C0959A01C09498C3
:100FE000789467C095FD0BC0F894B0937D00EAE655
:100FF000F0E0979862FF01C0C19A78945AC0F894C3
:10100000B0937D00E6E7F0E0979862FF01C0959A03
:1010100078944FC0B6E095FD07C0F894B0937D007A
:10102000949A9398789445C0F894B0937D00929ADE
:10103000939878943EC0B1E082FF24C095FD11C022
:1010400004E0F894B0937D00E0E9F0E00093B30091
:10105000C198929A62FF02C0959A01C094987894C0
:1010600028C001E0F894B0937D00ECE7F0E0009335
:10107000B3009598949A62FF02C0C19A01C09298F9
:10108000789417C095FD0BC0F894B0937D00E6E707
:10109000F0E0C19862FF01C0959A78940AC0F89474
:1010A000B0937D00EAE6F0E0959862FF01C0C19A36
:1010B00078946F7D089529E630E0F9012092B3001D
:1010C000C19897989598929A939A949A6B7F08955D
:1010D000A4EBB0E00FEF0D930D930D930D9303E090
:1010E0000D9304E00D9309E00D9303E00D9301E0EF
:1010F0000D9301E00D93A0ECB0E001E00D930FEF34
:101100000D930D930D930D930D9303E00D930FEF3E
:101110000D930FEF0D930D9305E20D9300ED0D93DD
:101120000AEF0D930AEF0D9304E00D930FEF0D936B
:1011300001E00D9300E00D930AE70D930FEF0D937F
:1011400000E00D9301E00D9300E00D9303E00D939B
:1011500008952091BB008B7F233009F48460B09107
:10116000BC00B33019F09F7DB1FD90629F7BB091C0
:10117000BD00B1FD9064223011F0886001C0877F0E
:1011800008950A95E00FF21DB4910895ECE1F0E0A6
:101190000091B400F6DFB093D800ECE1F0E00091EC
:1011A000B500EFDFB093D900EAE2F0E00091BA00B9
:1011B000E8DFB093DA00B091D0000FEF1CE0B2305E
:1011C00011F400EA1AE0B33011F402E815E00093DC
:1011D000720010937300E8E3F0E00091D700D1DFD4
:1011E000B093A200089508952091CA003091CB00D9
:1011F000B091BC00B33009F43E5097FF02C020E02C
:101200003FEFB32FB21B6B2EB25810F4B2E86B2E27
:1012100000E00395609EB12DBD57D8F30093AE005A
:1012200008959068E1DF0FDA20E030E0B0E16B2E46
:1012300006DAB09197002B0F321D6A94C9F7B4E01B
:1012400036952795BA95E1F7822E9F77CDDF0895E1
:10125000F894E3E0F0E0B9E0B7BFB491B078C1F33F
:10126000F894A895B1B5B861B1BDB0E0B1BDB4E036
:10127000BEBFBFE5BDBF1FDFB0E0B8BBB2E1B7BBCB
:10128000B0E0B5BBB0E0B4BBBCE1B2BBBCEBB1BB42
:101290002224A0E0B0E02D92AA31E9F7A0E6B0E068
:1012A0000FEF2D920A95E9F7B1E0B093A40010DF9B
:1012B000EDD2B6B1B460B6B90091CC000093AF00E6
:1012C000B1E0B0936A00F894C2D9CCD9BCD9CDD9D9
:1012D000BAD9CED9B8D961D3BAD9B9D9B6D9F894CF
:1012E0000AEF1AEFA6B396FDA095A0FF1FC01A95AE
:1012F000C9F70A95B1F7E0E0FCE1B591B43E39F4E5
:10130000B591B03E21F4B591BF3F09F40CC0E0E0C7
:10131000F395F395B591B83F49F4B591B43931F4EB
:10132000B591BA3A19F4EE27F695099412DF2EDF3B
:101330005ADF5ADF0091CC000093AF00BCDEB2E070
:10134000B3BFB2E0BEBDB2E0B5BDB1E5B8BFB9BF95
:10135000B0B7B77FB0BFB8B1B0B7B860B0BF6DD9E4
:101360007894FBDABEB5B06496FDBF7BBEBDB9B75D
:10137000B062B9BFBB27B062B8BF8D7F68D9626069
:1013800033E02CE0B0919600BB2321F42CE03A9599
:1013900009F4A5CF58D980FFA2CF8E7FB0919700D6
:1013A000B23078F3B92FBF71009199000093980083
:1013B000B0939900B01729F72A9521F76D7FBEB534
:1013C000B06496FDBF7BBEBDBB27B062B8BF8D7F4A
:1013D000B091D600BB2321F48062B92FB0709B2F4F
:1013E0008F7B2092670031D985FF05C0B0916700DF
:1013F000BA3008F0806423D902E085FF01C000E024
:10140000B0919700B017B8F3F8942CD92BD92AD9FA
:1014100078941DD920928700B091BC00B33009F4B4
:1014200074C00DD9B091C000B13008F46EC0B09155
:101430006A00B13008F469C085FD18C0B09197000A
:10144000BF3F08F462C0F89416D97894FED8B091E2
:101450009700B130C0F7F89405D9F3D803D9789440
:10146000F4D8B0919700BF3FB0F3C9C2B8E09B2E4B
:101470009068F894B9DE7894E8D8F8949F77B4DE51
:1014800080909700B0919700BF37789408F445C0DA
:10149000D4D8F894F0D878949A9451F7C2DEB82D45
:1014A000B550B093CB00D3D8F8941DD27BD27894AA
:1014B000BAE09B2E9068F89497DE7894C6D8F8949A
:1014C0009F7792DE80909700B0919700BF37789415
:1014D00078F7B3D8F894C6D8B4D8C4D878949A9486
:1014E00049F79FDEB82DBB5FB093CA00B0D8F8941F
:1014F000FAD167D27894A9D8F89476DE7894B0912E
:101500009700BF3F08F498CF7AC200919700B0913E
:1015100087000B1710F00093870097D801E0B09177
:10152000BC00B35009F405E0B0919700B01708F083
:1015300073CFF894A0D89FD89ED8789488D820925A
:101540006A0020926B0020926C00B0916B00B39502
:10155000B0936B00BF3F69F5B0916C00B395B09349
:101560006C00B091CE0009E1BA9559F002E3BA954A
:1015700041F00DE7BA9529F00AEFBA9511F02092E3
:101580006C00B0916C00B017A0F0B0916C00BA95EF
:10159000B0936C00B4EBB0936B00B091CD00B093FE
:1015A000AF00F89468D87894B091CC00B093AF00B5
:1015B0004CD847D8B0916800BB2319F485FF01C00F
:1015C0008ECE01E085FD01C006E0B0919700B01716
:1015D00008F4BBCFB091BC00B35009F036D8B0913D
:1015E0006800BB2309F47BCEF89465DD209261008E
:1015F0002092620020926300522C2092640020927C
:10160000A3007894B091B900BB0FB093A0002092D2
:101610007F00209280002092810020928200209200
:1016200083002092AC0060E070E020927100B8E08E
:10163000B093AC00786001D8B2E073FDB1E0B7B907
:10164000B6B1B068B064B6B9B6B1B6FDFDCF04B1FD
:1016500015B1B6B1BF77B6B9112309F00FEF0093FA
:10166000AD007DD9B8E0B093AC0078608090BB004D
:10167000B2E0B093BB006DDD8092BB00F894BFEF89
:10168000B0939C00B5D9B0916100B0939C00B09329
:101690009D00B0939E007894B1E0B0936100B09348
:1016A00063005B2EB0936400B093A600B0919B00E2
:1016B000B093A500B091BC00B33019F49F7D87FDB5
:1016C00090627160726020926D00A4DCB4DCA9D9D4
:1016D000AED9A7D9ACD9A5D906C0F8943ADD78948B
:1016E0002092AC00777F11DB3DD8C3DBF3DB9FD9C1
:1016F00005DB66FD38D876FFF0D876FD1ED9B9DB5C
:10170000FADB95D902DB66FD50D8B3DB33DC8FD929
:10171000F5DA66FD84D8ADDB3EDC89D9F6DA66FD04
:10172000AED8A7DB77DC83D9E9DAB2E073FDB1E0AC
:10173000B7B9B6B1B068B064B6B99BDB7CDC77D919
:101740000ED971FF23C067FD21C0B0919F00B093F7
:101750009C00B0939D00B0919B00B093A500B1E0B8
:10176000B093A60018E12CE0B0916D00B11740F0E5
:101770007D7F746020936F00BFEFB0939C0006C024
:10178000B0919700B13008F0AECF5AC072FF10C0D0
:1017900067FD0EC0B0916F00BA9511F47B7F9DCFAD
:1017A000B0936F00B0919700B13008F09CCF48C063
:1017B00020927000B0919A0002E8B01708F040C083
:1017C00085FF04C0B0916800BB23D1F1B091BC008B
:1017D000B33081F495FD03C087FD04C00BC087FFC3
:1017E00001C008C067FD06C06068B0919F00B0935B
:1017F0009C008ECF00EF67FF05C0B0919F00B093B3
:101800009C0000E2B0917B00B01708F46CCF67FF3A
:1018100017C06F779F7D87FD90627460B2E1B093CF
:101820006F00B0919F00B0939C005DCFB0917000AD
:10183000B395B0937000B0919700BB2309F002C03C
:1018400020927000F89437DC8090BB00B2E0B09337
:10185000BB007FDC8092BB0020926100209262007E
:1018600020926300522C209264002092A0007E7F80
:101870007894E3D620DCB6B1B460B6B985FF05C074
:10188000B0917000B53008F02ACD5BCEEDE0F0E00D
:1018900023D00A3509F01BC0EEE0F0E01DD0053A78
:1018A00009F015C03AE0A4EBB0E0E3E0F0E014D0BA
:1018B0000D9331963A95D9F738E1A0ECB0E0EFE01E
:1018C000F0E00AD00D9331963A95D9F702C000DCCA
:1018D0000AD0E7E2F0E00895E199FECFEEBBFFBB4E
:1018E000E09A0DB308951ED03AE0A4EBB0E0E3E037
:1018F000F0E00D910FD031963A95D9F738E1A0EC90
:10190000B0E0EFE0F0E00D9105D031963A95D9F7CF
:1019100012D00895E199FECF0DBBEEBBFFBBE29A5A
:10192000E19A0895EDE0F0E00FEFF4DFEEE0F0E093
:101930000FEFF0DF0895EDE0F0E00AE5EBDFEEE019
:10194000F0E005EAE7DF08953091B0000091B100C2
:10195000313011F40093B800323011F40093B90023
:10196000333011F40093BA00343011F40093C60000
:10197000353011F40093BB00363011F40093D700DA
:10198000373011F40093D000383011F40093BC00CC
:10199000393011F40093BD00089525E058D62A95FA
:1019A000E9F708955FD661D663D665D64AD65AD68A
:1019B0005CD65ED660D645D655D657D659D65BD6B8
:1019C000089559D655D651D64DD63BD654D650D675
:1019D0004CD648D636D64FD64BD647D643D60895A2
:1019E0008090B0009090B1003DD63CD63BD629D631
:1019F0008A94D1F740D625D69A94E1F70895F894C1
:101A0000D1DF7894CADFC9DFB1E0B093B000B1E0B4
:101A1000B093B1002092B200F894E2DF7894B5E080
:101A20006B2E7090970013D6B09197007B16C9F774
:101A3000B13018F0BF3F40F107C086DFF89453DFA4
:101A4000B1DFB8E0B1BDA9DF6A9459F7B091B20037
:101A5000B395B093B200B33008F4DECF9EDFB091FF
:101A6000B100B395B093B100F894B091B000BA95BD
:101A7000EEE3F0E0EB0FF21D049178940395B09142
:101A8000B100B01708F4C6CF88DF87DFB091B0008F
:101A9000B395B093B000B091B000BA3008F4B7CFAE
:0E1AA00017DBF89420DFB8E0B1BD77DFD1CBC3
:00000001FF
